 MFCN42UD

 Timestamp is 3588732f (Wed Jun 17 18:53:51 1998)

 Preferred load address is 5f600000

 Start         Length     Name                   Class
 0001:00000000 00000deaH .text                   CODE
 0001:00000df0 000003d7H .text$AFX_INIT          CODE
 0001:000011d0 00002313H .text$AFX_SOCK          CODE
 0001:000034f0 00000203H .text$AFX_VDEL          CODE
 0001:00003700 000000d4H .text$x                 CODE
 0002:00000000 00000248H .idata$5                DATA
 0002:00000250 000005ccH .rdata                  DATA
 0002:00000820 00000284H .rdata$r                DATA
 0002:00000aa8 000001a0H .xdata$x                DATA
 0002:00000c48 00000020H .didat$2                DATA
 0002:00000c68 00000020H .didat$3                DATA
 0002:00000c88 00000070H .didat$4                DATA
 0002:00000cf8 00000070H .didat$7                DATA
 0002:00000d68 00000050H .idata$2                DATA
 0002:00000db8 00000014H .idata$3                DATA
 0002:00000dcc 00000248H .idata$4                DATA
 0002:00001014 00000210H .idata$6                DATA
 0002:00001230 000001f1H .edata                  DATA
 0003:00000000 00000004H .CRT$XCA                DATA
 0003:00000004 00000004H .CRT$XCL                DATA
 0003:00000008 00000004H .CRT$XCZ                DATA
 0003:0000000c 00000004H .CRT$XIA                DATA
 0003:00000010 00000004H .CRT$XIZ                DATA
 0003:00000020 000001b0H .data                   DATA
 0003:000001d0 00000070H .didat$5                DATA
 0003:00000240 00000058H .bss                    DATA
 0004:00000000 00000058H .rsrc$01                DATA
 0004:00000060 00000368H .rsrc$02                DATA

  Address         Publics by Value              Rva+Base     Lib:Object

 0001:00000000       ?GetHead@CSimpleList@@QBEPAXXZ 5f601000 f i dllnet.obj
 0001:00000010       ??1CNoTrackObject@@UAE@XZ  5f601010 f i sockcore.obj
 0001:00000030       ??_ECNoTrackObject@@UAEPAXI@Z 5f601030 f i sockcore.obj
 0001:00000030       ??_GCNoTrackObject@@UAEPAXI@Z 5f601030 f i sockcore.obj
 0001:00000060       ?AtlW2AHelper@@YGPADPADPBGH@Z 5f601060 f i sockcore.obj
 0001:00000080       ?AtlW2AHelper@@YGPADPADPBGHI@Z 5f601080 f i sockcore.obj
 0001:0000010a       ?AfxGetModuleState@@YGPAVAFX_MODULE_STATE@@XZ 5f60110a f   MFC42UD:MFC42uD.DLL
 0001:00000110       ?AfxTermThread@@YGXPAUHINSTANCE__@@@Z 5f601110 f   MFC42UD:MFC42uD.DLL
 0001:00000116       ?AfxTermExtensionModule@@YGXAAUAFX_EXTENSION_MODULE@@H@Z 5f601116 f   MFC42UD:MFC42uD.DLL
 0001:0000011c       ??0CDynLinkLibrary@@QAE@AAUAFX_EXTENSION_MODULE@@H@Z 5f60111c f   MFC42UD:MFC42uD.DLL
 0001:00000122       ??2CObject@@SGPAXI@Z       5f601122 f   MFC42UD:MFC42uD.DLL
 0001:00000128       ?AfxAssertFailedLine@@YGHPBDH@Z 5f601128 f   MFC42UD:MFC42uD.DLL
 0001:0000012e       ?AfxInitExtensionModule@@YGHAAUAFX_EXTENSION_MODULE@@PAUHINSTANCE__@@@Z 5f60112e f   MFC42UD:MFC42uD.DLL
 0001:00000134       ??3CObject@@SGXPAX@Z       5f601134 f   MFC42UD:MFC42uD.DLL
 0001:0000013a       ?AfxGetAppModuleState@@YGPAVAFX_MODULE_STATE@@XZ 5f60113a f   MFC42UD:MFC42uD.DLL
 0001:00000140       ??3@YAXPAX@Z               5f601140 f   MFC42UD:MFC42uD.DLL
 0001:00000146       ??2@YAPAXI@Z               5f601146 f   MFC42UD:MFC42uD.DLL
 0001:0000014c       ??3CNoTrackObject@@SGXPAX@Z 5f60114c f   MFC42UD:MFC42uD.DLL
 0001:00000152       ?Serialize@CObject@@UAEXAAVCArchive@@@Z 5f601152 f   MFC42UD:MFC42uD.DLL
 0001:00000158       ??0CObject@@IAE@XZ         5f601158 f   MFC42UD:MFC42uD.DLL
 0001:0000015e       ??4CString@@QAEABV0@PBD@Z  5f60115e f   MFC42UD:MFC42uD.DLL
 0001:00000164       ?AfxGetModuleThreadState@@YGPAVAFX_MODULE_THREAD_STATE@@XZ 5f601164 f   MFC42UD:MFC42uD.DLL
 0001:0000016a       ??1CObject@@UAE@XZ         5f60116a f   MFC42UD:MFC42uD.DLL
 0001:00000170       ?GetValueAt@CMapPtrToPtr@@QBEPAXPAX@Z 5f601170 f   MFC42UD:MFC42uD.DLL
 0001:00000176       ??3CObject@@SGXPAXPBDH@Z   5f601176 f   MFC42UD:MFC42uD.DLL
 0001:0000017c       ?Lookup@CMapPtrToPtr@@QBEHPAXAAPAX@Z 5f60117c f   MFC42UD:MFC42uD.DLL
 0001:00000182       ?SetAt@CMapPtrToPtr@@QAEXPAX0@Z 5f601182 f   MFC42UD:MFC42uD.DLL
 0001:00000188       ?FromHandlePermanent@CWnd@@SGPAV1@PAUHWND__@@@Z 5f601188 f   MFC42UD:MFC42uD.DLL
 0001:0000018e       ?AfxThrowResourceException@@YGXXZ 5f60118e f   MFC42UD:MFC42uD.DLL
 0001:00000194       ?AfxTrace@@YAXPBGZZ        5f601194 f   MFC42UD:MFC42uD.DLL
 0001:0000019a       ?CreateEx@CWnd@@QAEHKPBG0KHHHHPAUHWND__@@PAUHMENU__@@PAX@Z 5f60119a f   MFC42UD:MFC42uD.DLL
 0001:000001a0       ?AfxRegisterWndClass@@YGPBGIPAUHICON__@@PAUHBRUSH__@@0@Z 5f6011a0 f   MFC42UD:MFC42uD.DLL
 0001:000001a6       ??2CObject@@SGPAXIPBDH@Z   5f6011a6 f   MFC42UD:MFC42uD.DLL
 0001:000001ac       ?IsEmpty@CMapPtrToPtr@@QBEHXZ 5f6011ac f   MFC42UD:MFC42uD.DLL
 0001:000001b2       ?AfxEnableMemoryTracking@@YGHH@Z 5f6011b2 f   MFC42UD:MFC42uD.DLL
 0001:000001b8       ?RemoveHead@CPtrList@@QAEPAXXZ 5f6011b8 f   MFC42UD:MFC42uD.DLL
 0001:000001be       ?IsEmpty@CPtrList@@QBEHXZ  5f6011be f   MFC42UD:MFC42uD.DLL
 0001:000001c4       ?RemoveAll@CMapPtrToPtr@@QAEXXZ 5f6011c4 f   MFC42UD:MFC42uD.DLL
 0001:000001ca       ?AfxAssertValidObject@@YGXPBVCObject@@PBDH@Z 5f6011ca f   MFC42UD:MFC42uD.DLL
 0001:000001d0       ?RemoveKey@CMapPtrToPtr@@QAEHPAX@Z 5f6011d0 f   MFC42UD:MFC42uD.DLL
 0001:000001d6       ?AssertValid@CObject@@UBEXXZ 5f6011d6 f   MFC42UD:MFC42uD.DLL
 0001:000001dc       ??6CDumpContext@@QAEAAV0@I@Z 5f6011dc f   MFC42UD:MFC42uD.DLL
 0001:000001e2       ??6CDumpContext@@QAEAAV0@PBD@Z 5f6011e2 f   MFC42UD:MFC42uD.DLL
 0001:000001e8       ?Dump@CObject@@UBEXAAVCDumpContext@@@Z 5f6011e8 f   MFC42UD:MFC42uD.DLL
 0001:000001ee       ?AddTail@CPtrList@@QAEPAU__POSITION@@PAX@Z 5f6011ee f   MFC42UD:MFC42uD.DLL
 0001:000001f4       ??2@YAPAXIPBDH@Z           5f6011f4 f   MFC42UD:MFC42uD.DLL
 0001:000001fa       ?Delete@CException@@QAEXXZ 5f6011fa f   MFC42UD:MFC42uD.DLL
 0001:00000200       ?IsKindOf@CObject@@QBEHPBUCRuntimeClass@@@Z 5f601200 f   MFC42UD:MFC42uD.DLL
 0001:00000206       ?AfxGetThread@@YGPAVCWinThread@@XZ 5f601206 f   MFC42UD:MFC42uD.DLL
 0001:0000020c       ??6CDumpContext@@QAEAAV0@H@Z 5f60120c f   MFC42UD:MFC42uD.DLL
 0001:00000212       ??6CDumpContext@@QAEAAV0@PBX@Z 5f601212 f   MFC42UD:MFC42uD.DLL
 0001:00000218       ?GetBufferPtr@CFile@@UAEIIIPAPAX0@Z 5f601218 f   MFC42UD:MFC42uD.DLL
 0001:0000021e       ?SetFilePath@CFile@@UAEXPBG@Z 5f60121e f   MFC42UD:MFC42uD.DLL
 0001:00000224       ?GetFilePath@CFile@@UBE?AVCString@@XZ 5f601224 f   MFC42UD:MFC42uD.DLL
 0001:0000022a       ?GetFileTitle@CFile@@UBE?AVCString@@XZ 5f60122a f   MFC42UD:MFC42uD.DLL
 0001:00000230       ?GetFileName@CFile@@UBE?AVCString@@XZ 5f601230 f   MFC42UD:MFC42uD.DLL
 0001:00000236       ??1CFile@@UAE@XZ           5f601236 f   MFC42UD:MFC42uD.DLL
 0001:0000023c       ??0CFile@@QAE@XZ           5f60123c f   MFC42UD:MFC42uD.DLL
 0001:00000242       ?AfxThrowFileException@@YGXHJPBG@Z 5f601242 f   MFC42UD:MFC42uD.DLL
 0001:00000248       ?AfxThrowNotSupportedException@@YGXXZ 5f601248 f   MFC42UD:MFC42uD.DLL
 0001:0000024e       ?AssertValid@CFile@@UBEXXZ 5f60124e f   MFC42UD:MFC42uD.DLL
 0001:00000254       ??6CDumpContext@@QAEAAV0@PBVCObject@@@Z 5f601254 f   MFC42UD:MFC42uD.DLL
 0001:0000025a       ?GetDepth@CDumpContext@@QBEHXZ 5f60125a f   MFC42UD:MFC42uD.DLL
 0001:00000260       ?Dump@CFile@@UBEXAAVCDumpContext@@@Z 5f601260 f   MFC42UD:MFC42uD.DLL
 0001:00000266       ?SetOccDialogInfo@CWnd@@MAEHPAU_AFX_OCC_DIALOG_INFO@@@Z 5f601266 f   MFC42UD:MFC42uD.DLL
 0001:0000026c       ?IsFrameWnd@CWnd@@UBEHXZ   5f60126c f   MFC42UD:MFC42uD.DLL
 0001:00000272       ?CheckAutoCenter@CWnd@@UAEHXZ 5f601272 f   MFC42UD:MFC42uD.DLL
 0001:00000278       ?OnChildNotify@CWnd@@MAEHIIJPAJ@Z 5f601278 f   MFC42UD:MFC42uD.DLL
 0001:0000027e       ?PostNcDestroy@CWnd@@MAEXXZ 5f60127e f   MFC42UD:MFC42uD.DLL
 0001:00000284       ?DefWindowProcW@CWnd@@MAEJIIJ@Z 5f601284 f   MFC42UD:MFC42uD.DLL
 0001:0000028a       ?OnWndMsg@CWnd@@MAEHIIJPAJ@Z 5f60128a f   MFC42UD:MFC42uD.DLL
 0001:00000290       ?WindowProc@CWnd@@MAEJIIJ@Z 5f601290 f   MFC42UD:MFC42uD.DLL
 0001:00000296       ?OnAmbientProperty@CWnd@@UAEHPAVCOleControlSite@@JPAUtagVARIANT@@@Z 5f601296 f   MFC42UD:MFC42uD.DLL
 0001:0000029c       ?PreTranslateMessage@CWnd@@UAEHPAUtagMSG@@@Z 5f60129c f   MFC42UD:MFC42uD.DLL
 0001:000002a2       ?EndModalState@CWnd@@UAEXXZ 5f6012a2 f   MFC42UD:MFC42uD.DLL
 0001:000002a8       ?BeginModalState@CWnd@@UAEXXZ 5f6012a8 f   MFC42UD:MFC42uD.DLL
 0001:000002ae       ?DoDataExchange@CWnd@@MAEXPAVCDataExchange@@@Z 5f6012ae f   MFC42UD:MFC42uD.DLL
 0001:000002b4       ?GetSuperWndProcAddr@CWnd@@MAEPAP6GJPAUHWND__@@IIJ@ZXZ 5f6012b4 f   MFC42UD:MFC42uD.DLL
 0001:000002ba       ?OnNotify@CWnd@@MAEHIJPAJ@Z 5f6012ba f   MFC42UD:MFC42uD.DLL
 0001:000002c0       ?OnCommand@CWnd@@MAEHIJ@Z  5f6012c0 f   MFC42UD:MFC42uD.DLL
 0001:000002c6       ?EndModalLoop@CWnd@@UAEXH@Z 5f6012c6 f   MFC42UD:MFC42uD.DLL
 0001:000002cc       ?ContinueModal@CWnd@@UAEHXZ 5f6012cc f   MFC42UD:MFC42uD.DLL
 0001:000002d2       ?WinHelpW@CWnd@@UAEXKI@Z   5f6012d2 f   MFC42UD:MFC42uD.DLL
 0001:000002d8       ?GetScrollBarCtrl@CWnd@@UBEPAVCScrollBar@@H@Z 5f6012d8 f   MFC42UD:MFC42uD.DLL
 0001:000002de       ?OnToolHitTest@CWnd@@UBEHVCPoint@@PAUtagTOOLINFOW@@@Z 5f6012de f   MFC42UD:MFC42uD.DLL
 0001:000002e4       ?CalcWindowRect@CWnd@@UAEXPAUtagRECT@@I@Z 5f6012e4 f   MFC42UD:MFC42uD.DLL
 0001:000002ea       ?PreCreateWindow@CWnd@@UAEHAAUtagCREATESTRUCTW@@@Z 5f6012ea f   MFC42UD:MFC42uD.DLL
 0001:000002f0       ?DestroyWindow@CWnd@@UAEHXZ 5f6012f0 f   MFC42UD:MFC42uD.DLL
 0001:000002f6       ?Create@CWnd@@UAEHPBG0KABUtagRECT@@PAV1@IPAUCCreateContext@@@Z 5f6012f6 f   MFC42UD:MFC42uD.DLL
 0001:000002fc       ?PreSubclassWindow@CWnd@@UAEXXZ 5f6012fc f   MFC42UD:MFC42uD.DLL
 0001:00000302       ?GetConnectionHook@CCmdTarget@@MAEPAUIConnectionPoint@@ABU_GUID@@@Z 5f601302 f   MFC42UD:MFC42uD.DLL
 0001:00000308       ?GetExtraConnectionPoints@CCmdTarget@@MAEHPAVCPtrArray@@@Z 5f601308 f   MFC42UD:MFC42uD.DLL
 0001:0000030e       ?GetInterfaceHook@CCmdTarget@@UAEPAUIUnknown@@PBX@Z 5f60130e f   MFC42UD:MFC42uD.DLL
 0001:00000314       ?OnCreateAggregates@CCmdTarget@@UAEHXZ 5f601314 f   MFC42UD:MFC42uD.DLL
 0001:0000031a       ?GetEventSinkMap@CCmdTarget@@MBEPBUAFX_EVENTSINKMAP@@XZ 5f60131a f   MFC42UD:MFC42uD.DLL
 0001:00000320       ?GetInterfaceMap@CCmdTarget@@MBEPBUAFX_INTERFACEMAP@@XZ 5f601320 f   MFC42UD:MFC42uD.DLL
 0001:00000326       ?GetConnectionMap@CCmdTarget@@MBEPBUAFX_CONNECTIONMAP@@XZ 5f601326 f   MFC42UD:MFC42uD.DLL
 0001:0000032c       ?GetDispatchMap@CCmdTarget@@MBEPBUAFX_DISPMAP@@XZ 5f60132c f   MFC42UD:MFC42uD.DLL
 0001:00000332       ?GetCommandMap@CCmdTarget@@MBEPBUAFX_OLECMDMAP@@XZ 5f601332 f   MFC42UD:MFC42uD.DLL
 0001:00000338       ?GetTypeLib@CCmdTarget@@UAEJKPAPAUITypeLib@@@Z 5f601338 f   MFC42UD:MFC42uD.DLL
 0001:0000033e       ?GetTypeLibCache@CCmdTarget@@UAEPAVCTypeLibCache@@XZ 5f60133e f   MFC42UD:MFC42uD.DLL
 0001:00000344       ?GetTypeInfoCount@CCmdTarget@@UAEIXZ 5f601344 f   MFC42UD:MFC42uD.DLL
 0001:0000034a       ?GetDispatchIID@CCmdTarget@@UAEHPAU_GUID@@@Z 5f60134a f   MFC42UD:MFC42uD.DLL
 0001:00000350       ?IsInvokeAllowed@CCmdTarget@@UAEHJ@Z 5f601350 f   MFC42UD:MFC42uD.DLL
 0001:00000356       ?OnFinalRelease@CWnd@@UAEXXZ 5f601356 f   MFC42UD:MFC42uD.DLL
 0001:0000035c       ?OnCmdMsg@CCmdTarget@@UAEHIHPAXPAUAFX_CMDHANDLERINFO@@@Z 5f60135c f   MFC42UD:MFC42uD.DLL
 0001:00000362       ?Dump@CWnd@@UBEXAAVCDumpContext@@@Z 5f601362 f   MFC42UD:MFC42uD.DLL
 0001:00000368       ?AssertValid@CWnd@@UBEXXZ  5f601368 f   MFC42UD:MFC42uD.DLL
 0001:0000036e       ?GetRuntimeClass@CWnd@@UBEPAUCRuntimeClass@@XZ 5f60136e f   MFC42UD:MFC42uD.DLL
 0001:00000374       ??0CWnd@@QAE@XZ            5f601374 f   MFC42UD:MFC42uD.DLL
 0001:0000037a       ??1CWnd@@UAE@XZ            5f60137a f   MFC42UD:MFC42uD.DLL
 0001:00000380       ??1CProcessLocalObject@@QAE@XZ 5f601380 f   MFC42UD:MFC42uD.DLL
 0001:00000386       ?GetData@CProcessLocalObject@@QAEPAVCNoTrackObject@@P6GPAV2@XZ@Z 5f601386 f   MFC42UD:MFC42uD.DLL
 0001:0000038c       ??2CNoTrackObject@@SGPAXI@Z 5f60138c f   MFC42UD:MFC42uD.DLL
 0001:00000392       ___CxxFrameHandler         5f601392 f   msvcrtd:MSVCRTD.dll
 0001:000003a0       ??_L@YGXPAXIHP6EX0@Z1@Z    5f6013a0 f   msvcrtd:ehvecctr.obj
 0001:00000440       ??_M@YGXPAXIHP6EX0@Z@Z     5f601440 f   msvcrtd:ehvecdtr.obj
 0001:000004f0       ?__ArrayUnwind@@YGXPAXIHP6EX0@Z@Z 5f6014f0 f   msvcrtd:ehvecdtr.obj
 0001:000005a0       ??0type_info@@AAE@ABV0@@Z  5f6015a0 f   msvcrtd:ti_inst.obj
 0001:000005c0       ??_Etype_info@@UAEPAXI@Z   5f6015c0 f i msvcrtd:ti_inst.obj
 0001:000005c0       ??_Gtype_info@@UAEPAXI@Z   5f6015c0 f i msvcrtd:ti_inst.obj
 0001:000005f0       ??4type_info@@AAEAAV0@ABV0@@Z 5f6015f0 f   msvcrtd:ti_inst.obj
 0001:00000600       _memset                    5f601600 f   msvcrtd:MSVCRTD.dll
 0001:00000610       __chkstk                   5f601610 f   msvcrtd:chkstk.obj
 0001:00000610       __alloca_probe             5f601610 f   msvcrtd:chkstk.obj
 0001:00000640       __CrtDbgReport             5f601640 f   msvcrtd:MSVCRTD.dll
 0001:00000650       __onexit                   5f601650 f   msvcrtd:atonexit.obj
 0001:00000690       _atexit                    5f601690 f   msvcrtd:atonexit.obj
 0001:000006b0       __CRT_INIT@12              5f6016b0 f   msvcrtd:crtdll.obj
 0001:000007c0       __DllMainCRTStartup@12     5f6017c0 f   msvcrtd:crtdll.obj
 0001:000008b4       __except_handler3          5f6018b4 f   msvcrtd:MSVCRTD.dll
 0001:000008ba       ?terminate@@YAXXZ          5f6018ba f   msvcrtd:MSVCRTD.dll
 0001:000008c0       ??1type_info@@UAE@XZ       5f6018c0 f   msvcrtd:MSVCRTD.dll
 0001:000008c6       ___dllonexit               5f6018c6 f   msvcrtd:MSVCRTD.dll
 0001:000008cc       __free_dbg                 5f6018cc f   msvcrtd:MSVCRTD.dll
 0001:000008d2       __initterm                 5f6018d2 f   msvcrtd:MSVCRTD.dll
 0001:000008d8       __malloc_dbg               5f6018d8 f   msvcrtd:MSVCRTD.dll
 0001:000008de       _FreeLibrary@4             5f6018de f   kernel32:KERNEL32.dll
 0001:000008e4       _GetModuleHandleA@4        5f6018e4 f   kernel32:KERNEL32.dll
 0001:000008ea       _LocalFree@4               5f6018ea f   kernel32:KERNEL32.dll
 0001:000008f0       _LocalAlloc@8              5f6018f0 f   kernel32:KERNEL32.dll
 0001:000008f6       _LoadLibraryA@4            5f6018f6 f   kernel32:KERNEL32.dll
 0001:000008fc       _SetLastError@4            5f6018fc f   kernel32:KERNEL32.dll
 0001:00000902       _lstrlenW@4                5f601902 f   kernel32:KERNEL32.dll
 0001:00000908       _WideCharToMultiByte@32    5f601908 f   kernel32:KERNEL32.dll
 0001:0000090e       _PostMessageW@16           5f60190e f   user32:USER32.dll
 0001:00000914       _DispatchMessageW@4        5f601914 f   user32:USER32.dll
 0001:0000091a       _PeekMessageW@20           5f60191a f   user32:USER32.dll
 0001:00000920       _KillTimer@8               5f601920 f   user32:USER32.dll
 0001:00000926       _WaitMessage@0             5f601926 f   user32:USER32.dll
 0001:0000092c       _SetTimer@16               5f60192c f   user32:USER32.dll
 0001:00000932       __imp_load__WSACleanup@0   5f601932     wsock32:WSOCK32.dll
 0001:0000093e       __tailMerge_WSOCK32        5f60193e     wsock32:WSOCK32.dll
 0001:0000094c       _WSACleanup@0              5f60194c     wsock32:WSOCK32.dll
 0001:00000952       __imp_load__WSAStartup@8   5f601952     wsock32:WSOCK32.dll
 0001:0000095e       _WSAStartup@8              5f60195e     wsock32:WSOCK32.dll
 0001:00000964       __imp_load__WSASetLastError@4 5f601964     wsock32:WSOCK32.dll
 0001:00000970       _WSASetLastError@4         5f601970     wsock32:WSOCK32.dll
 0001:00000976       __imp_load__inet_ntoa@4    5f601976     wsock32:WSOCK32.dll
 0001:00000982       _inet_ntoa@4               5f601982     wsock32:WSOCK32.dll
 0001:00000988       __imp_load__ntohs@4        5f601988     wsock32:WSOCK32.dll
 0001:00000994       _ntohs@4                   5f601994     wsock32:WSOCK32.dll
 0001:0000099a       __imp_load__accept@12      5f60199a     wsock32:WSOCK32.dll
 0001:000009a6       _accept@12                 5f6019a6     wsock32:WSOCK32.dll
 0001:000009ac       __imp_load__htons@4        5f6019ac     wsock32:WSOCK32.dll
 0001:000009b8       _htons@4                   5f6019b8     wsock32:WSOCK32.dll
 0001:000009be       __imp_load__inet_addr@4    5f6019be     wsock32:WSOCK32.dll
 0001:000009ca       _inet_addr@4               5f6019ca     wsock32:WSOCK32.dll
 0001:000009d0       __imp_load__htonl@4        5f6019d0     wsock32:WSOCK32.dll
 0001:000009dc       _htonl@4                   5f6019dc     wsock32:WSOCK32.dll
 0001:000009e2       __imp_load__closesocket@4  5f6019e2     wsock32:WSOCK32.dll
 0001:000009ee       _closesocket@4             5f6019ee     wsock32:WSOCK32.dll
 0001:000009f4       __imp_load__gethostbyname@4 5f6019f4     wsock32:WSOCK32.dll
 0001:00000a00       _gethostbyname@4           5f601a00     wsock32:WSOCK32.dll
 0001:00000a06       __imp_load__recv@16        5f601a06     wsock32:WSOCK32.dll
 0001:00000a12       _recv@16                   5f601a12     wsock32:WSOCK32.dll
 0001:00000a18       __imp_load__send@16        5f601a18     wsock32:WSOCK32.dll
 0001:00000a24       _send@16                   5f601a24     wsock32:WSOCK32.dll
 0001:00000a2a       __imp_load__WSAAsyncSelect@16 5f601a2a     wsock32:WSOCK32.dll
 0001:00000a36       _WSAAsyncSelect@16         5f601a36     wsock32:WSOCK32.dll
 0001:00000a3c       __imp_load__WSAGetLastError@0 5f601a3c     wsock32:WSOCK32.dll
 0001:00000a48       _WSAGetLastError@0         5f601a48     wsock32:WSOCK32.dll
 0001:00000a4e       __imp_load__socket@12      5f601a4e     wsock32:WSOCK32.dll
 0001:00000a5a       _socket@12                 5f601a5a     wsock32:WSOCK32.dll
 0001:00000a60       __imp_load__recvfrom@24    5f601a60     wsock32:WSOCK32.dll
 0001:00000a6c       _recvfrom@24               5f601a6c     wsock32:WSOCK32.dll
 0001:00000a72       __imp_load__sendto@24      5f601a72     wsock32:WSOCK32.dll
 0001:00000a7e       _sendto@24                 5f601a7e     wsock32:WSOCK32.dll
 0001:00000a84       __imp_load__connect@12     5f601a84     wsock32:WSOCK32.dll
 0001:00000a90       _connect@12                5f601a90     wsock32:WSOCK32.dll
 0001:00000a96       __imp_load__getpeername@12 5f601a96     wsock32:WSOCK32.dll
 0001:00000aa2       _getpeername@12            5f601aa2     wsock32:WSOCK32.dll
 0001:00000aa8       __imp_load__getsockname@12 5f601aa8     wsock32:WSOCK32.dll
 0001:00000ab4       _getsockname@12            5f601ab4     wsock32:WSOCK32.dll
 0001:00000aba       __imp_load__setsockopt@20  5f601aba     wsock32:WSOCK32.dll
 0001:00000ac6       _setsockopt@20             5f601ac6     wsock32:WSOCK32.dll
 0001:00000acc       __imp_load__getsockopt@20  5f601acc     wsock32:WSOCK32.dll
 0001:00000ad8       _getsockopt@20             5f601ad8     wsock32:WSOCK32.dll
 0001:00000ade       __imp_load__bind@12        5f601ade     wsock32:WSOCK32.dll
 0001:00000aea       _bind@12                   5f601aea     wsock32:WSOCK32.dll
 0001:00000af0       __imp_load__ioctlsocket@12 5f601af0     wsock32:WSOCK32.dll
 0001:00000afc       _ioctlsocket@12            5f601afc     wsock32:WSOCK32.dll
 0001:00000b02       __imp_load__listen@8       5f601b02     wsock32:WSOCK32.dll
 0001:00000b0e       _listen@8                  5f601b0e     wsock32:WSOCK32.dll
 0001:00000b14       __imp_load__shutdown@8     5f601b14     wsock32:WSOCK32.dll
 0001:00000b20       _shutdown@8                5f601b20     wsock32:WSOCK32.dll
 0001:00000b26       ___delayLoadHelper@8       5f601b26 f   delayimp:delayhlp.obj
 0001:00000d1f       ___FUnloadDelayLoadedDLL@4 5f601d1f f   delayimp:delayhlp.obj
 0001:00000dd2       _GetProcAddress@8          5f601dd2 f   kernel32:KERNEL32.dll
 0001:00000dd8       _InterlockedExchange@8     5f601dd8 f   kernel32:KERNEL32.dll
 0001:00000dde       _RaiseException@16         5f601dde f   kernel32:KERNEL32.dll
 0001:00000de4       _GetLastError@0            5f601de4 f   kernel32:KERNEL32.dll
 0001:00000df0       _RawDllMain@12             5f601df0 f   dllnet.obj
 0001:00000e8e       _DllMain@12                5f601e8e f   dllnet.obj
 0001:00000f4d       ?AfxNetInitModule@@YGXXZ   5f601f4d f   dllnet.obj
 0001:00001010       ?_GetBaseClass@CAsyncSocket@@KGPAUCRuntimeClass@@XZ 5f602010 f   sockcore.obj
 0001:0000101a       ?GetRuntimeClass@CAsyncSocket@@UBEPAUCRuntimeClass@@XZ 5f60201a f   sockcore.obj
 0001:0000102a       ?_GetBaseClass@CSocket@@KGPAUCRuntimeClass@@XZ 5f60202a f   sockcore.obj
 0001:00001034       ?GetRuntimeClass@CSocket@@UBEPAUCRuntimeClass@@XZ 5f602034 f   sockcore.obj
 0001:00001044       ?_GetBaseClass@CSocketFile@@KGPAUCRuntimeClass@@XZ 5f602044 f   sockcore.obj
 0001:0000104e       ?GetRuntimeClass@CSocketFile@@UBEPAUCRuntimeClass@@XZ 5f60204e f   sockcore.obj
 0001:000010a0       ??1?$CProcessLocal@V_AFX_SOCK_STATE@@@@QAE@XZ 5f6020a0 f i sockcore.obj
 0001:000010c0       ??C?$CEmbeddedButActsLikePtr@VCMapPtrToPtr@@@@QAEPAVCMapPtrToPtr@@XZ 5f6020c0 f i sockcore.obj
 0001:000010c0       ??C?$CEmbeddedButActsLikePtr@VCPtrList@@@@QAEPAVCPtrList@@XZ 5f6020c0 f i sockcore.obj
 0001:000010d0       ?GetData@?$CProcessLocal@V_AFX_SOCK_STATE@@@@QAEPAV_AFX_SOCK_STATE@@XZ 5f6020d0 f i sockcore.obj
 0001:00001120       ?CreateObject@?$CProcessLocal@V_AFX_SOCK_STATE@@@@SGPAVCNoTrackObject@@XZ 5f602120 f i sockcore.obj
 0001:00001190       ??0_AFX_SOCK_STATE@@QAE@XZ 5f602190 f i sockcore.obj
 0001:000011b0       ??0CNoTrackObject@@QAE@XZ  5f6021b0 f i sockcore.obj
 0001:000011d0       ??1_AFX_SOCK_STATE@@UAE@XZ 5f6021d0 f   sockcore.obj
 0001:00001228       ?AfxSocketTerm@@YGXXZ      5f602228 f   sockcore.obj
 0001:0000126b       ?AfxSocketInit@@YGHPAUWSAData@@@Z 5f60226b f   sockcore.obj
 0001:0000130c       ??0CAsyncSocket@@QAE@XZ    5f60230c f   sockcore.obj
 0001:00001335       ?Create@CAsyncSocket@@QAEHIHJPBG@Z 5f602335 f   sockcore.obj
 0001:00001395       ?Attach@CAsyncSocket@@QAEHIJ@Z 5f602395 f   sockcore.obj
 0001:000013e9       ?Detach@CAsyncSocket@@QAEIXZ 5f6023e9 f   sockcore.obj
 0001:0000142c       ?GetPeerName@CAsyncSocket@@QAEHAAVCString@@AAI@Z 5f60242c f   sockcore.obj
 0001:00001494       ?GetSockName@CAsyncSocket@@QAEHAAVCString@@AAI@Z 5f602494 f   sockcore.obj
 0001:000014fc       ?Accept@CAsyncSocket@@UAEHAAV1@PAUsockaddr@@PAH@Z 5f6024fc f   sockcore.obj
 0001:000015e4       ?Bind@CAsyncSocket@@QAEHIPBG@Z 5f6025e4 f   sockcore.obj
 0001:000016cc       ?Close@CAsyncSocket@@UAEXXZ 5f6026cc f   sockcore.obj
 0001:0000172b       ?Connect@CAsyncSocket@@QAEHPBGI@Z 5f60272b f   sockcore.obj
 0001:00001842       ?Receive@CAsyncSocket@@UAEHPAXHH@Z 5f602842 f   sockcore.obj
 0001:00001867       ?ReceiveFrom@CAsyncSocket@@QAEHPAXHAAVCString@@AAIH@Z 5f602867 f   sockcore.obj
 0001:000018db       ?Send@CAsyncSocket@@UAEHPBXHH@Z 5f6028db f   sockcore.obj
 0001:00001900       ?SendTo@CAsyncSocket@@QAEHPBXHIPBGH@Z 5f602900 f   sockcore.obj
 0001:00001a10       ?AsyncSelect@CAsyncSocket@@QAEHJ@Z 5f602a10 f   sockcore.obj
 0001:00001a99       ?OnReceive@CAsyncSocket@@MAEXH@Z 5f602a99 f   sockcore.obj
 0001:00001aa6       ?OnSend@CAsyncSocket@@MAEXH@Z 5f602aa6 f   sockcore.obj
 0001:00001ab3       ?OnOutOfBandData@CAsyncSocket@@MAEXH@Z 5f602ab3 f   sockcore.obj
 0001:00001ac0       ?OnAccept@CAsyncSocket@@MAEXH@Z 5f602ac0 f   sockcore.obj
 0001:00001acd       ?OnConnect@CAsyncSocket@@MAEXH@Z 5f602acd f   sockcore.obj
 0001:00001ada       ?OnClose@CAsyncSocket@@MAEXH@Z 5f602ada f   sockcore.obj
 0001:00001ae7       ??1CAsyncSocket@@UAE@XZ    5f602ae7 f   sockcore.obj
 0001:00001b41       ?LookupHandle@CAsyncSocket@@SGPAV1@IH@Z 5f602b41 f   sockcore.obj
 0001:00001ba7       ?AttachHandle@CAsyncSocket@@SGXIPAV1@H@Z 5f602ba7 f   sockcore.obj
 0001:00001def       ?DetachHandle@CAsyncSocket@@SGXIH@Z 5f602def f   sockcore.obj
 0001:00001f9f       ?KillSocket@CAsyncSocket@@SGXIPAV1@@Z 5f602f9f f   sockcore.obj
 0001:0000201b       ?DoCallBack@CAsyncSocket@@SGXIJ@Z 5f60301b f   sockcore.obj
 0001:000021c9       ?Socket@CAsyncSocket@@QAEHHJHH@Z 5f6031c9 f   sockcore.obj
 0001:00002241       ?AssertValid@CAsyncSocket@@UBEXXZ 5f603241 f   sockcore.obj
 0001:0000228d       ?Dump@CAsyncSocket@@UBEXAAVCDumpContext@@@Z 5f60328d f   sockcore.obj
 0001:000022e6       ?ReceiveFromHelper@CAsyncSocket@@MAEHPAXHPAUsockaddr@@PAHH@Z 5f6032e6 f   sockcore.obj
 0001:00002313       ?SendToHelper@CAsyncSocket@@MAEHPBXHPBUsockaddr@@HH@Z 5f603313 f   sockcore.obj
 0001:00002340       ?ConnectHelper@CAsyncSocket@@MAEHPBUsockaddr@@H@Z 5f603340 f   sockcore.obj
 0001:0000236b       ??0CSocket@@QAE@XZ         5f60336b f   sockcore.obj
 0001:000023a8       ?CancelBlockingCall@CSocket@@QAEXXZ 5f6033a8 f   sockcore.obj
 0001:000023d2       ?OnMessagePending@CSocket@@MAEHXZ 5f6033d2 f   sockcore.obj
 0001:00002405       ??1CSocket@@UAE@XZ         5f603405 f   sockcore.obj
 0001:0000245f       ?Accept@CSocket@@UAEHAAVCAsyncSocket@@PAUsockaddr@@PAH@Z 5f60345f f   sockcore.obj
 0001:000024c9       ?Close@CSocket@@UAEXXZ     5f6034c9 f   sockcore.obj
 0001:00002525       ?Receive@CSocket@@UAEHPAXHH@Z 5f603525 f   sockcore.obj
 0001:00002596       ?Send@CSocket@@UAEHPBXHH@Z 5f603596 f   sockcore.obj
 0001:0000260a       ?SendChunk@CSocket@@QAEHPBXHH@Z 5f60360a f   sockcore.obj
 0001:00002664       ?ConnectHelper@CSocket@@MAEHPBUsockaddr@@H@Z 5f603664 f   sockcore.obj
 0001:000026f3       ?ReceiveFromHelper@CSocket@@MAEHPAXHPAUsockaddr@@PAHH@Z 5f6036f3 f   sockcore.obj
 0001:0000276c       ?SendToHelper@CSocket@@MAEHPBXHPBUsockaddr@@HH@Z 5f60376c f   sockcore.obj
 0001:000027e6       ?ProcessAuxQueue@CSocket@@SGHXZ 5f6037e6 f   sockcore.obj
 0001:000028ef       ?AuxQueueAdd@CSocket@@KGXIIJ@Z 5f6038ef f   sockcore.obj
 0001:00002951       ?PumpMessages@CSocket@@MAEHI@Z 5f603951 f   sockcore.obj
 0001:00002c11       ?AssertValid@CSocket@@MBEXXZ 5f603c11 f   sockcore.obj
 0001:00002c24       ?Dump@CSocket@@MBEXAAVCDumpContext@@@Z 5f603c24 f   sockcore.obj
 0001:00002c8b       ??0CSocketFile@@QAE@PAVCSocket@@H@Z 5f603c8b f   sockcore.obj
 0001:00002da5       ??1CSocketFile@@UAE@XZ     5f603da5 f   sockcore.obj
 0001:00002dc1       ?Read@CSocketFile@@UAEIPAXI@Z 5f603dc1 f   sockcore.obj
 0001:00002f06       ?Write@CSocketFile@@UAEXPBXI@Z 5f603f06 f   sockcore.obj
 0001:00002f77       ?Close@CSocketFile@@UAEXXZ 5f603f77 f   sockcore.obj
 0001:00002f8c       ?Open@CSocketFile@@UAEHPBGIPAVCFileException@@@Z 5f603f8c f   sockcore.obj
 0001:00002fa0       ?Duplicate@CSocketFile@@UBEPAVCFile@@XZ 5f603fa0 f   sockcore.obj
 0001:00002fb2       ?GetPosition@CSocketFile@@UBEKXZ 5f603fb2 f   sockcore.obj
 0001:00002fc4       ?Seek@CSocketFile@@UAEJJI@Z 5f603fc4 f   sockcore.obj
 0001:00002ff1       ?SetLength@CSocketFile@@UAEXK@Z 5f603ff1 f   sockcore.obj
 0001:00003003       ?GetLength@CSocketFile@@UBEKXZ 5f604003 f   sockcore.obj
 0001:00003015       ?LockRange@CSocketFile@@UAEXKK@Z 5f604015 f   sockcore.obj
 0001:00003027       ?UnlockRange@CSocketFile@@UAEXKK@Z 5f604027 f   sockcore.obj
 0001:00003039       ?Flush@CSocketFile@@UAEXXZ 5f604039 f   sockcore.obj
 0001:00003044       ?Abort@CSocketFile@@UAEXXZ 5f604044 f   sockcore.obj
 0001:00003054       ?AssertValid@CSocketFile@@UBEXXZ 5f604054 f   sockcore.obj
 0001:00003086       ?Dump@CSocketFile@@UBEXAAVCDumpContext@@@Z 5f604086 f   sockcore.obj
 0001:000030de       ??0CSocketWnd@@QAE@XZ      5f6040de f   sockcore.obj
 0001:000030fd       ?OnSocketNotify@CSocketWnd@@IAEJIJ@Z 5f6040fd f   sockcore.obj
 0001:00003123       ?OnSocketDead@CSocketWnd@@IAEJIJ@Z 5f604123 f   sockcore.obj
 0001:00003149       ?_GetBaseMessageMap@CSocketWnd@@KGPBUAFX_MSGMAP@@XZ 5f604149 f   sockcore.obj
 0001:00003153       ?GetMessageMap@CSocketWnd@@MBEPBUAFX_MSGMAP@@XZ 5f604153 f   sockcore.obj
 0001:00003163       ??BCAsyncSocket@@QBEIXZ    5f604163 f   sockcore.obj
 0001:00003174       ?GetPeerName@CAsyncSocket@@QAEHPAUsockaddr@@PAH@Z 5f604174 f   sockcore.obj
 0001:0000319f       ?GetSockName@CAsyncSocket@@QAEHPAUsockaddr@@PAH@Z 5f60419f f   sockcore.obj
 0001:000031ca       ?SetSockOpt@CAsyncSocket@@QAEHHPBXHH@Z 5f6041ca f   sockcore.obj
 0001:000031fd       ?GetSockOpt@CAsyncSocket@@QAEHHPAXPAHH@Z 5f6041fd f   sockcore.obj
 0001:00003230       ?FromHandle@CAsyncSocket@@SGPAV1@I@Z 5f604230 f   sockcore.obj
 0001:00003242       ?GetLastError@CAsyncSocket@@SGHXZ 5f604242 f   sockcore.obj
 0001:0000324c       ?Bind@CAsyncSocket@@QAEHPBUsockaddr@@H@Z 5f60424c f   sockcore.obj
 0001:00003277       ?Connect@CAsyncSocket@@QAEHPBUsockaddr@@H@Z 5f604277 f   sockcore.obj
 0001:00003297       ?IOCtl@CAsyncSocket@@QAEHJPAK@Z 5f604297 f   sockcore.obj
 0001:000032c2       ?Listen@CAsyncSocket@@QAEHH@Z 5f6042c2 f   sockcore.obj
 0001:000032e9       ?ReceiveFrom@CAsyncSocket@@QAEHPAXHPAUsockaddr@@PAHH@Z 5f6042e9 f   sockcore.obj
 0001:00003315       ?ShutDown@CAsyncSocket@@QAEHH@Z 5f604315 f   sockcore.obj
 0001:0000333c       ?SendTo@CAsyncSocket@@QAEHPBXHPBUsockaddr@@HH@Z 5f60433c f   sockcore.obj
 0001:00003368       ?Create@CSocket@@QAEHIHPBG@Z 5f604368 f   sockcore.obj
 0001:0000338b       ?IsBlocking@CSocket@@QAEHXZ 5f60438b f   sockcore.obj
 0001:000033a4       ?FromHandle@CSocket@@SGPAV1@I@Z 5f6043a4 f   sockcore.obj
 0001:000033b6       ?Attach@CSocket@@QAEHI@Z   5f6043b6 f   sockcore.obj
 0001:000033e0       ??_G_AFX_SOCK_STATE@@UAEPAXI@Z 5f6043e0 f i sockcore.obj
 0001:000033e0       ??_E_AFX_SOCK_STATE@@UAEPAXI@Z 5f6043e0 f i sockcore.obj
 0001:00003410       ??_GCAsyncSocket@@UAEPAXI@Z 5f604410 f i sockcore.obj
 0001:00003440       ??_GCSocket@@UAEPAXI@Z     5f604440 f i sockcore.obj
 0001:00003470       ??_GCSocketFile@@UAEPAXI@Z 5f604470 f i sockcore.obj
 0001:00003470       ??_ECSocketFile@@UAEPAXI@Z 5f604470 f i sockcore.obj
 0001:000034a0       ??_ECSocketWnd@@UAEPAXI@Z  5f6044a0 f i sockcore.obj
 0001:000034a0       ??_GCSocketWnd@@UAEPAXI@Z  5f6044a0 f i sockcore.obj
 0001:000034d0       ??1CSocketWnd@@UAE@XZ      5f6044d0 f i sockcore.obj
 0001:00003600       ??_ECAsyncSocket@@UAEPAXI@Z 5f604600 f i dllnet.obj
 0001:00003670       ??_ECSocket@@UAEPAXI@Z     5f604670 f i dllnet.obj
 0001:000036e0       ??B?$CTypedSimpleList@PAUCRuntimeClass@@@@QAEPAUCRuntimeClass@@XZ 5f6046e0 f i dllnet.obj
 0001:000036e0       ??B?$CTypedSimpleList@PAVCOleObjectFactory@@@@QAEPAVCOleObjectFactory@@XZ 5f6046e0 f i dllnet.obj
 0002:00000000       __imp__FreeLibrary@4       5f605000     kernel32:KERNEL32.dll
 0002:00000004       __imp__GetModuleHandleA@4  5f605004     kernel32:KERNEL32.dll
 0002:00000008       __imp__LocalFree@4         5f605008     kernel32:KERNEL32.dll
 0002:0000000c       __imp__LocalAlloc@8        5f60500c     kernel32:KERNEL32.dll
 0002:00000010       __imp__LoadLibraryA@4      5f605010     kernel32:KERNEL32.dll
 0002:00000014       __imp__SetLastError@4      5f605014     kernel32:KERNEL32.dll
 0002:00000018       __imp__lstrlenW@4          5f605018     kernel32:KERNEL32.dll
 0002:0000001c       __imp__WideCharToMultiByte@32 5f60501c     kernel32:KERNEL32.dll
 0002:00000020       __imp__GetProcAddress@8    5f605020     kernel32:KERNEL32.dll
 0002:00000024       __imp__InterlockedExchange@8 5f605024     kernel32:KERNEL32.dll
 0002:00000028       __imp__RaiseException@16   5f605028     kernel32:KERNEL32.dll
 0002:0000002c       __imp__GetLastError@0      5f60502c     kernel32:KERNEL32.dll
 0002:00000030       \177KERNEL32_NULL_THUNK_DATA 5f605030     kernel32:KERNEL32.dll
 0002:00000034       __imp_??4CString@@QAEABV0@PBD@Z 5f605034     MFC42UD:MFC42uD.DLL
 0002:00000038       __imp_?AfxGetModuleThreadState@@YGPAVAFX_MODULE_THREAD_STATE@@XZ 5f605038     MFC42UD:MFC42uD.DLL
 0002:0000003c       __imp_??1CObject@@UAE@XZ   5f60503c     MFC42UD:MFC42uD.DLL
 0002:00000040       __imp_?GetValueAt@CMapPtrToPtr@@QBEPAXPAX@Z 5f605040     MFC42UD:MFC42uD.DLL
 0002:00000044       __imp_??0CObject@@IAE@XZ   5f605044     MFC42UD:MFC42uD.DLL
 0002:00000048       __imp_??3CObject@@SGXPAXPBDH@Z 5f605048     MFC42UD:MFC42uD.DLL
 0002:0000004c       __imp_?Lookup@CMapPtrToPtr@@QBEHPAXAAPAX@Z 5f60504c     MFC42UD:MFC42uD.DLL
 0002:00000050       __imp_?SetAt@CMapPtrToPtr@@QAEXPAX0@Z 5f605050     MFC42UD:MFC42uD.DLL
 0002:00000054       __imp_?FromHandlePermanent@CWnd@@SGPAV1@PAUHWND__@@@Z 5f605054     MFC42UD:MFC42uD.DLL
 0002:00000058       __imp_?AfxThrowResourceException@@YGXXZ 5f605058     MFC42UD:MFC42uD.DLL
 0002:0000005c       __imp_?AfxTrace@@YAXPBGZZ  5f60505c     MFC42UD:MFC42uD.DLL
 0002:00000060       __imp_?CreateEx@CWnd@@QAEHKPBG0KHHHHPAUHWND__@@PAUHMENU__@@PAX@Z 5f605060     MFC42UD:MFC42uD.DLL
 0002:00000064       __imp_?AfxRegisterWndClass@@YGPBGIPAUHICON__@@PAUHBRUSH__@@0@Z 5f605064     MFC42UD:MFC42uD.DLL
 0002:00000068       __imp_??2CObject@@SGPAXIPBDH@Z 5f605068     MFC42UD:MFC42uD.DLL
 0002:0000006c       __imp_?IsEmpty@CMapPtrToPtr@@QBEHXZ 5f60506c     MFC42UD:MFC42uD.DLL
 0002:00000070       __imp_?AfxEnableMemoryTracking@@YGHH@Z 5f605070     MFC42UD:MFC42uD.DLL
 0002:00000074       __imp_?RemoveHead@CPtrList@@QAEPAXXZ 5f605074     MFC42UD:MFC42uD.DLL
 0002:00000078       __imp_?IsEmpty@CPtrList@@QBEHXZ 5f605078     MFC42UD:MFC42uD.DLL
 0002:0000007c       __imp_?RemoveAll@CMapPtrToPtr@@QAEXXZ 5f60507c     MFC42UD:MFC42uD.DLL
 0002:00000080       __imp_?AfxAssertValidObject@@YGXPBVCObject@@PBDH@Z 5f605080     MFC42UD:MFC42uD.DLL
 0002:00000084       __imp_?RemoveKey@CMapPtrToPtr@@QAEHPAX@Z 5f605084     MFC42UD:MFC42uD.DLL
 0002:00000088       __imp_?AssertValid@CObject@@UBEXXZ 5f605088     MFC42UD:MFC42uD.DLL
 0002:0000008c       __imp_??6CDumpContext@@QAEAAV0@I@Z 5f60508c     MFC42UD:MFC42uD.DLL
 0002:00000090       __imp_??6CDumpContext@@QAEAAV0@PBD@Z 5f605090     MFC42UD:MFC42uD.DLL
 0002:00000094       __imp_?Dump@CObject@@UBEXAAVCDumpContext@@@Z 5f605094     MFC42UD:MFC42uD.DLL
 0002:00000098       __imp_?AddTail@CPtrList@@QAEPAU__POSITION@@PAX@Z 5f605098     MFC42UD:MFC42uD.DLL
 0002:0000009c       __imp_??2@YAPAXIPBDH@Z     5f60509c     MFC42UD:MFC42uD.DLL
 0002:000000a0       __imp_?Delete@CException@@QAEXXZ 5f6050a0     MFC42UD:MFC42uD.DLL
 0002:000000a4       __imp_?IsKindOf@CObject@@QBEHPBUCRuntimeClass@@@Z 5f6050a4     MFC42UD:MFC42uD.DLL
 0002:000000a8       __imp_?classCException@CException@@2UCRuntimeClass@@B 5f6050a8     MFC42UD:MFC42uD.DLL
 0002:000000ac       __imp_?AfxGetThread@@YGPAVCWinThread@@XZ 5f6050ac     MFC42UD:MFC42uD.DLL
 0002:000000b0       __imp_??6CDumpContext@@QAEAAV0@H@Z 5f6050b0     MFC42UD:MFC42uD.DLL
 0002:000000b4       __imp_??6CDumpContext@@QAEAAV0@PBX@Z 5f6050b4     MFC42UD:MFC42uD.DLL
 0002:000000b8       __imp_?GetBufferPtr@CFile@@UAEIIIPAPAX0@Z 5f6050b8     MFC42UD:MFC42uD.DLL
 0002:000000bc       __imp_?SetFilePath@CFile@@UAEXPBG@Z 5f6050bc     MFC42UD:MFC42uD.DLL
 0002:000000c0       __imp_?GetFilePath@CFile@@UBE?AVCString@@XZ 5f6050c0     MFC42UD:MFC42uD.DLL
 0002:000000c4       __imp_?GetFileTitle@CFile@@UBE?AVCString@@XZ 5f6050c4     MFC42UD:MFC42uD.DLL
 0002:000000c8       __imp_?GetFileName@CFile@@UBE?AVCString@@XZ 5f6050c8     MFC42UD:MFC42uD.DLL
 0002:000000cc       __imp_??1CFile@@UAE@XZ     5f6050cc     MFC42UD:MFC42uD.DLL
 0002:000000d0       __imp_??0CFile@@QAE@XZ     5f6050d0     MFC42UD:MFC42uD.DLL
 0002:000000d4       __imp_?AfxThrowFileException@@YGXHJPBG@Z 5f6050d4     MFC42UD:MFC42uD.DLL
 0002:000000d8       __imp_?AfxThrowNotSupportedException@@YGXXZ 5f6050d8     MFC42UD:MFC42uD.DLL
 0002:000000dc       __imp_?AssertValid@CFile@@UBEXXZ 5f6050dc     MFC42UD:MFC42uD.DLL
 0002:000000e0       __imp_??6CDumpContext@@QAEAAV0@PBVCObject@@@Z 5f6050e0     MFC42UD:MFC42uD.DLL
 0002:000000e4       __imp_?GetDepth@CDumpContext@@QBEHXZ 5f6050e4     MFC42UD:MFC42uD.DLL
 0002:000000e8       __imp_?Dump@CFile@@UBEXAAVCDumpContext@@@Z 5f6050e8     MFC42UD:MFC42uD.DLL
 0002:000000ec       __imp_?SetOccDialogInfo@CWnd@@MAEHPAU_AFX_OCC_DIALOG_INFO@@@Z 5f6050ec     MFC42UD:MFC42uD.DLL
 0002:000000f0       __imp_?IsFrameWnd@CWnd@@UBEHXZ 5f6050f0     MFC42UD:MFC42uD.DLL
 0002:000000f4       __imp_?CheckAutoCenter@CWnd@@UAEHXZ 5f6050f4     MFC42UD:MFC42uD.DLL
 0002:000000f8       __imp_??3CNoTrackObject@@SGXPAX@Z 5f6050f8     MFC42UD:MFC42uD.DLL
 0002:000000fc       __imp_?Serialize@CObject@@UAEXAAVCArchive@@@Z 5f6050fc     MFC42UD:MFC42uD.DLL
 0002:00000100       __imp_?DefWindowProcW@CWnd@@MAEJIIJ@Z 5f605100     MFC42UD:MFC42uD.DLL
 0002:00000104       __imp_?OnWndMsg@CWnd@@MAEHIIJPAJ@Z 5f605104     MFC42UD:MFC42uD.DLL
 0002:00000108       __imp_?WindowProc@CWnd@@MAEJIIJ@Z 5f605108     MFC42UD:MFC42uD.DLL
 0002:0000010c       __imp_?OnAmbientProperty@CWnd@@UAEHPAVCOleControlSite@@JPAUtagVARIANT@@@Z 5f60510c     MFC42UD:MFC42uD.DLL
 0002:00000110       __imp_?PreTranslateMessage@CWnd@@UAEHPAUtagMSG@@@Z 5f605110     MFC42UD:MFC42uD.DLL
 0002:00000114       __imp_?EndModalState@CWnd@@UAEXXZ 5f605114     MFC42UD:MFC42uD.DLL
 0002:00000118       __imp_?BeginModalState@CWnd@@UAEXXZ 5f605118     MFC42UD:MFC42uD.DLL
 0002:0000011c       __imp_?DoDataExchange@CWnd@@MAEXPAVCDataExchange@@@Z 5f60511c     MFC42UD:MFC42uD.DLL
 0002:00000120       __imp_?GetSuperWndProcAddr@CWnd@@MAEPAP6GJPAUHWND__@@IIJ@ZXZ 5f605120     MFC42UD:MFC42uD.DLL
 0002:00000124       __imp_?AfxGetModuleState@@YGPAVAFX_MODULE_STATE@@XZ 5f605124     MFC42UD:MFC42uD.DLL
 0002:00000128       __imp_?OnCommand@CWnd@@MAEHIJ@Z 5f605128     MFC42UD:MFC42uD.DLL
 0002:0000012c       __imp_?EndModalLoop@CWnd@@UAEXH@Z 5f60512c     MFC42UD:MFC42uD.DLL
 0002:00000130       __imp_?ContinueModal@CWnd@@UAEHXZ 5f605130     MFC42UD:MFC42uD.DLL
 0002:00000134       __imp_?WinHelpW@CWnd@@UAEXKI@Z 5f605134     MFC42UD:MFC42uD.DLL
 0002:00000138       __imp_?GetScrollBarCtrl@CWnd@@UBEPAVCScrollBar@@H@Z 5f605138     MFC42UD:MFC42uD.DLL
 0002:0000013c       __imp_?OnToolHitTest@CWnd@@UBEHVCPoint@@PAUtagTOOLINFOW@@@Z 5f60513c     MFC42UD:MFC42uD.DLL
 0002:00000140       __imp_?CalcWindowRect@CWnd@@UAEXPAUtagRECT@@I@Z 5f605140     MFC42UD:MFC42uD.DLL
 0002:00000144       __imp_?PreCreateWindow@CWnd@@UAEHAAUtagCREATESTRUCTW@@@Z 5f605144     MFC42UD:MFC42uD.DLL
 0002:00000148       __imp_?DestroyWindow@CWnd@@UAEHXZ 5f605148     MFC42UD:MFC42uD.DLL
 0002:0000014c       __imp_?Create@CWnd@@UAEHPBG0KABUtagRECT@@PAV1@IPAUCCreateContext@@@Z 5f60514c     MFC42UD:MFC42uD.DLL
 0002:00000150       __imp_?PreSubclassWindow@CWnd@@UAEXXZ 5f605150     MFC42UD:MFC42uD.DLL
 0002:00000154       __imp_?GetConnectionHook@CCmdTarget@@MAEPAUIConnectionPoint@@ABU_GUID@@@Z 5f605154     MFC42UD:MFC42uD.DLL
 0002:00000158       __imp_?GetExtraConnectionPoints@CCmdTarget@@MAEHPAVCPtrArray@@@Z 5f605158     MFC42UD:MFC42uD.DLL
 0002:0000015c       __imp_?GetInterfaceHook@CCmdTarget@@UAEPAUIUnknown@@PBX@Z 5f60515c     MFC42UD:MFC42uD.DLL
 0002:00000160       __imp_?OnCreateAggregates@CCmdTarget@@UAEHXZ 5f605160     MFC42UD:MFC42uD.DLL
 0002:00000164       __imp_?GetEventSinkMap@CCmdTarget@@MBEPBUAFX_EVENTSINKMAP@@XZ 5f605164     MFC42UD:MFC42uD.DLL
 0002:00000168       __imp_?GetInterfaceMap@CCmdTarget@@MBEPBUAFX_INTERFACEMAP@@XZ 5f605168     MFC42UD:MFC42uD.DLL
 0002:0000016c       __imp_?GetConnectionMap@CCmdTarget@@MBEPBUAFX_CONNECTIONMAP@@XZ 5f60516c     MFC42UD:MFC42uD.DLL
 0002:00000170       __imp_?GetDispatchMap@CCmdTarget@@MBEPBUAFX_DISPMAP@@XZ 5f605170     MFC42UD:MFC42uD.DLL
 0002:00000174       __imp_?GetCommandMap@CCmdTarget@@MBEPBUAFX_OLECMDMAP@@XZ 5f605174     MFC42UD:MFC42uD.DLL
 0002:00000178       __imp_?GetTypeLib@CCmdTarget@@UAEJKPAPAUITypeLib@@@Z 5f605178     MFC42UD:MFC42uD.DLL
 0002:0000017c       __imp_?GetTypeLibCache@CCmdTarget@@UAEPAVCTypeLibCache@@XZ 5f60517c     MFC42UD:MFC42uD.DLL
 0002:00000180       __imp_?GetTypeInfoCount@CCmdTarget@@UAEIXZ 5f605180     MFC42UD:MFC42uD.DLL
 0002:00000184       __imp_?GetDispatchIID@CCmdTarget@@UAEHPAU_GUID@@@Z 5f605184     MFC42UD:MFC42uD.DLL
 0002:00000188       __imp_?IsInvokeAllowed@CCmdTarget@@UAEHJ@Z 5f605188     MFC42UD:MFC42uD.DLL
 0002:0000018c       __imp_?OnFinalRelease@CWnd@@UAEXXZ 5f60518c     MFC42UD:MFC42uD.DLL
 0002:00000190       __imp_?OnCmdMsg@CCmdTarget@@UAEHIHPAXPAUAFX_CMDHANDLERINFO@@@Z 5f605190     MFC42UD:MFC42uD.DLL
 0002:00000194       __imp_?Dump@CWnd@@UBEXAAVCDumpContext@@@Z 5f605194     MFC42UD:MFC42uD.DLL
 0002:00000198       __imp_?AssertValid@CWnd@@UBEXXZ 5f605198     MFC42UD:MFC42uD.DLL
 0002:0000019c       __imp_?GetRuntimeClass@CWnd@@UBEPAUCRuntimeClass@@XZ 5f60519c     MFC42UD:MFC42uD.DLL
 0002:000001a0       __imp_??0CWnd@@QAE@XZ      5f6051a0     MFC42UD:MFC42uD.DLL
 0002:000001a4       __imp_??1CWnd@@UAE@XZ      5f6051a4     MFC42UD:MFC42uD.DLL
 0002:000001a8       __imp_?messageMap@CWnd@@1UAFX_MSGMAP@@B 5f6051a8     MFC42UD:MFC42uD.DLL
 0002:000001ac       __imp_?classCObject@CObject@@2UCRuntimeClass@@B 5f6051ac     MFC42UD:MFC42uD.DLL
 0002:000001b0       __imp_?classCFile@CFile@@2UCRuntimeClass@@B 5f6051b0     MFC42UD:MFC42uD.DLL
 0002:000001b4       __imp_??1CProcessLocalObject@@QAE@XZ 5f6051b4     MFC42UD:MFC42uD.DLL
 0002:000001b8       __imp_?GetData@CProcessLocalObject@@QAEPAVCNoTrackObject@@P6GPAV2@XZ@Z 5f6051b8     MFC42UD:MFC42uD.DLL
 0002:000001bc       __imp_??2CNoTrackObject@@SGPAXI@Z 5f6051bc     MFC42UD:MFC42uD.DLL
 0002:000001c0       __imp_??2@YAPAXI@Z         5f6051c0     MFC42UD:MFC42uD.DLL
 0002:000001c4       __imp_??3@YAXPAX@Z         5f6051c4     MFC42UD:MFC42uD.DLL
 0002:000001c8       __imp_?AfxGetAppModuleState@@YGPAVAFX_MODULE_STATE@@XZ 5f6051c8     MFC42UD:MFC42uD.DLL
 0002:000001cc       __imp_??3CObject@@SGXPAX@Z 5f6051cc     MFC42UD:MFC42uD.DLL
 0002:000001d0       __imp_?AfxInitExtensionModule@@YGHAAUAFX_EXTENSION_MODULE@@PAUHINSTANCE__@@@Z 5f6051d0     MFC42UD:MFC42uD.DLL
 0002:000001d4       __imp_?AfxAssertFailedLine@@YGHPBDH@Z 5f6051d4     MFC42UD:MFC42uD.DLL
 0002:000001d8       __imp_??2CObject@@SGPAXI@Z 5f6051d8     MFC42UD:MFC42uD.DLL
 0002:000001dc       __imp_??0CDynLinkLibrary@@QAE@AAUAFX_EXTENSION_MODULE@@H@Z 5f6051dc     MFC42UD:MFC42uD.DLL
 0002:000001e0       __imp_?AfxTermExtensionModule@@YGXAAUAFX_EXTENSION_MODULE@@H@Z 5f6051e0     MFC42UD:MFC42uD.DLL
 0002:000001e4       __imp_?AfxTermThread@@YGXPAUHINSTANCE__@@@Z 5f6051e4     MFC42UD:MFC42uD.DLL
 0002:000001e8       __imp_?PostNcDestroy@CWnd@@MAEXXZ 5f6051e8     MFC42UD:MFC42uD.DLL
 0002:000001ec       __imp_?OnChildNotify@CWnd@@MAEHIIJPAJ@Z 5f6051ec     MFC42UD:MFC42uD.DLL
 0002:000001f0       __imp_?OnNotify@CWnd@@MAEHIJPAJ@Z 5f6051f0     MFC42UD:MFC42uD.DLL
 0002:000001f4       \177MFC42uD_NULL_THUNK_DATA 5f6051f4     MFC42UD:MFC42uD.DLL
 0002:000001f8       __imp____CxxFrameHandler   5f6051f8     msvcrtd:MSVCRTD.dll
 0002:000001fc       __imp___adjust_fdiv        5f6051fc     msvcrtd:MSVCRTD.dll
 0002:00000200       __imp___malloc_dbg         5f605200     msvcrtd:MSVCRTD.dll
 0002:00000204       __imp___initterm           5f605204     msvcrtd:MSVCRTD.dll
 0002:00000208       __imp___free_dbg           5f605208     msvcrtd:MSVCRTD.dll
 0002:0000020c       __imp___onexit             5f60520c     msvcrtd:MSVCRTD.dll
 0002:00000210       __imp____dllonexit         5f605210     msvcrtd:MSVCRTD.dll
 0002:00000214       __imp_??1type_info@@UAE@XZ 5f605214     msvcrtd:MSVCRTD.dll
 0002:00000218       __imp_?terminate@@YAXXZ    5f605218     msvcrtd:MSVCRTD.dll
 0002:0000021c       __imp__memset              5f60521c     msvcrtd:MSVCRTD.dll
 0002:00000220       __imp___except_handler3    5f605220     msvcrtd:MSVCRTD.dll
 0002:00000224       __imp___CrtDbgReport       5f605224     msvcrtd:MSVCRTD.dll
 0002:00000228       \177MSVCRTD_NULL_THUNK_DATA 5f605228     msvcrtd:MSVCRTD.dll
 0002:0000022c       __imp__SetTimer@16         5f60522c     user32:USER32.dll
 0002:00000230       __imp__WaitMessage@0       5f605230     user32:USER32.dll
 0002:00000234       __imp__KillTimer@8         5f605234     user32:USER32.dll
 0002:00000238       __imp__PeekMessageW@20     5f605238     user32:USER32.dll
 0002:0000023c       __imp__PostMessageW@16     5f60523c     user32:USER32.dll
 0002:00000240       __imp__DispatchMessageW@4  5f605240     user32:USER32.dll
 0002:00000244       \177USER32_NULL_THUNK_DATA 5f605244     user32:USER32.dll
 0002:00000270       _IID_IDocHostUIHandlerDispatch 5f605270     dllnet.obj
 0002:00000280       _IID_IInternalConnection   5f605280     dllnet.obj
 0002:00000290       _IID_IAxWinAmbientDispatch 5f605290     dllnet.obj
 0002:000002a0       _IID_IAxWinHostWindow      5f6052a0     dllnet.obj
 0002:000002b0       _IID_IRegistrar            5f6052b0     dllnet.obj
 0002:000002c0       _CLSID_Registrar           5f6052c0     dllnet.obj
 0002:000002d0       _LIBID_ATLLib              5f6052d0     dllnet.obj
 0002:000002e0       ??_C@_0M@IGON@MFC42UD?4DLL?$AA@ 5f6052e0     dllnet.obj
 0002:000002f0       ?classCSocketFile@CSocketFile@@2UCRuntimeClass@@B 5f6052f0     sockcore.obj
 0002:00000308       ??_C@_0M@FJKI@CSocketFile?$AA@ 5f605308     sockcore.obj
 0002:00000318       ?classCSocket@CSocket@@2UCRuntimeClass@@B 5f605318     sockcore.obj
 0002:00000330       ??_C@_07MBCI@CSocket?$AA@  5f605330     sockcore.obj
 0002:00000338       ?classCAsyncSocket@CAsyncSocket@@2UCRuntimeClass@@B 5f605338     sockcore.obj
 0002:00000350       ??_C@_0N@CCKH@CAsyncSocket?$AA@ 5f605350     sockcore.obj
 0002:00000360       ?messageMap@CSocketWnd@@1UAFX_MSGMAP@@B 5f605360     sockcore.obj
 0002:00000368       ?_messageEntries@CSocketWnd@@0QBUAFX_MSGMAP_ENTRY@@B 5f605368     sockcore.obj
 0002:000003b4       ??_7_AFX_SOCK_STATE@@6B@   5f6053b4     sockcore.obj
 0002:000003bc       ??_7CAsyncSocket@@6B@      5f6053bc     sockcore.obj
 0002:00000408       ??_7CNoTrackObject@@6B@    5f605408     sockcore.obj
 0002:0000040c       ??_C@_15DEDE@?$AA?$CF?$AAs?$AA?$AA@ 5f60540c     sockcore.obj
 0002:00000414       ??_C@_1GC@LFCO@?$AAW?$AAa?$AAr?$AAn?$AAi?$AAn?$AAg?$AA?3?$AA?5?$AAu?$AAn?$AAa?$AAb?$AAl?$AAe?$AA?5?$AAt?$AAo?$AA?5?$AAc@ 5f605414     sockcore.obj
 0002:00000478       ??_C@_1DC@CDHD@?$AAS?$AAo?$AAc?$AAk?$AAe?$AAt?$AA?5?$AAN?$AAo?$AAt?$AAi?$AAf?$AAi?$AAc?$AAa?$AAt?$AAi?$AAo?$AAn?$AA?5@ 5f605478     sockcore.obj
 0002:000004ac       ??_C@_08PEKM@lpa?5?$CB?$DN?50?$AA@ 5f6054ac     sockcore.obj
 0002:000004b8       ??_C@_0CH@IIKL@E?3?28168?2vc98?2mfc?2atl?2include?2atl@ 5f6054b8     sockcore.obj
 0002:000004e0       ??_C@_08NDGO@lpw?5?$CB?$DN?50?$AA@ 5f6054e0     sockcore.obj
 0002:000004ec       ??_C@_01BJG@?6?$AA@        5f6054ec     sockcore.obj
 0002:000004f0       ??_C@_0BA@MMD@INVALID_SOCKET?6?$AA@ 5f6054f0     sockcore.obj
 0002:00000500       ??_C@_0N@HJN@m_hSocket?5?$DN?5?$AA@ 5f605500     sockcore.obj
 0002:00000514       ??_7CSocket@@6B@           5f605514     sockcore.obj
 0002:00000564       ??_C@_1GM@FHGK@?$AAE?$AAr?$AAr?$AAo?$AAr?$AA?3?$AA?5?$AAc?$AAa?$AAu?$AAg?$AAh?$AAt?$AA?5?$AAe?$AAx?$AAc?$AAe?$AAp?$AAt@ 5f605564     sockcore.obj
 0002:000005d0       ??_C@_0BD@MNOG@m_nConnectError?5?$DN?5?$AA@ 5f6055d0     sockcore.obj
 0002:000005e4       ??_C@_0BA@EKGE@m_pbBlocking?5?$DN?5?$AA@ 5f6055e4     sockcore.obj
 0002:000005f8       ??_7CSocketFile@@6B@       5f6055f8     sockcore.obj
 0002:00000654       ??_C@_1GC@HBBN@?$AAW?$AAa?$AAr?$AAn?$AAi?$AAn?$AAg?$AA?5?$AA?9?$AA?5?$AAA?$AAt?$AAt?$AAe?$AAm?$AAp?$AAt?$AA?5?$AAm?$AAa@ 5f605654     sockcore.obj
 0002:000006b8       ??_C@_0O@FJPJ@with?5socket?3?5?$AA@ 5f6056b8     sockcore.obj
 0002:000006c8       ??_C@_0BA@JPDC@with?5no?5socket?6?$AA@ 5f6056c8     sockcore.obj
 0002:000006dc       ??_7CSocketWnd@@6B@        5f6056dc     sockcore.obj
 0002:0000079c       ??_C@_0CH@KFAI@E?3?28168?2vc98?2mfc?2mfc?2include?2afx@ 5f60579c     sockcore.obj
 0002:000007f8       ??_7type_info@@6B@         5f6057f8     msvcrtd:ti_inst.obj
 0002:000007fc       ??_C@_08JKC@crtdll?4c?$AA@ 5f6057fc     msvcrtd:crtdll.obj
 0002:00000810       __sz_WSOCK32               5f605810     wsock32:WSOCK32.dll
 0002:00000820       ??_R1A@?0A@A@CNoTrackObject@@8 5f605820     sockcore.obj
 0002:00000838       ??_R1A@?0A@A@_AFX_SOCK_STATE@@8 5f605838     sockcore.obj
 0002:00000850       ??_R2_AFX_SOCK_STATE@@8    5f605850     sockcore.obj
 0002:00000860       ??_R3_AFX_SOCK_STATE@@8    5f605860     sockcore.obj
 0002:00000870       ??_R4_AFX_SOCK_STATE@@6B@  5f605870     sockcore.obj
 0002:00000888       ??_R1A@?0A@A@CObject@@8    5f605888     sockcore.obj
 0002:000008a0       ??_R1A@?0A@A@CAsyncSocket@@8 5f6058a0     sockcore.obj
 0002:000008b8       ??_R2CAsyncSocket@@8       5f6058b8     sockcore.obj
 0002:000008c8       ??_R3CAsyncSocket@@8       5f6058c8     sockcore.obj
 0002:000008d8       ??_R4CAsyncSocket@@6B@     5f6058d8     sockcore.obj
 0002:000008ec       ??_R2CNoTrackObject@@8     5f6058ec     sockcore.obj
 0002:000008f8       ??_R3CNoTrackObject@@8     5f6058f8     sockcore.obj
 0002:00000908       ??_R4CNoTrackObject@@6B@   5f605908     sockcore.obj
 0002:00000920       ??_R1A@?0A@A@CSocket@@8    5f605920     sockcore.obj
 0002:00000938       ??_R2CSocket@@8            5f605938     sockcore.obj
 0002:00000948       ??_R3CSocket@@8            5f605948     sockcore.obj
 0002:00000958       ??_R4CSocket@@6B@          5f605958     sockcore.obj
 0002:00000970       ??_R1A@?0A@A@CFile@@8      5f605970     sockcore.obj
 0002:00000988       ??_R1A@?0A@A@CSocketFile@@8 5f605988     sockcore.obj
 0002:000009a0       ??_R2CSocketFile@@8        5f6059a0     sockcore.obj
 0002:000009b0       ??_R3CSocketFile@@8        5f6059b0     sockcore.obj
 0002:000009c0       ??_R4CSocketFile@@6B@      5f6059c0     sockcore.obj
 0002:000009d8       ??_R1A@?0A@A@CCmdTarget@@8 5f6059d8     sockcore.obj
 0002:000009f0       ??_R1A@?0A@A@CWnd@@8       5f6059f0     sockcore.obj
 0002:00000a08       ??_R1A@?0A@A@CSocketWnd@@8 5f605a08     sockcore.obj
 0002:00000a20       ??_R2CSocketWnd@@8         5f605a20     sockcore.obj
 0002:00000a38       ??_R3CSocketWnd@@8         5f605a38     sockcore.obj
 0002:00000a48       ??_R4CSocketWnd@@6B@       5f605a48     sockcore.obj
 0002:00000a60       ??_R1A@?0A@A@type_info@@8  5f605a60     msvcrtd:ti_inst.obj
 0002:00000a78       ??_R2type_info@@8          5f605a78     msvcrtd:ti_inst.obj
 0002:00000a80       ??_R3type_info@@8          5f605a80     msvcrtd:ti_inst.obj
 0002:00000a90       ??_R4type_info@@6B@        5f605a90     msvcrtd:ti_inst.obj
 0002:00000c48       __DELAY_IMPORT_DESCRIPTOR_WSOCK32 5f605c48     wsock32:WSOCK32.dll
 0002:00000c68       __NULL_DELAY_IMPORT_DESCRIPTOR 5f605c68     wsock32:WSOCK32.dll
 0002:00000cf4       \177WSOCK32_NULL_THUNK_DATA_DLN 5f605cf4     wsock32:WSOCK32.dll
 0002:00000cfc       \177WSOCK32_NULL_THUNK_DATA_DLB 5f605cfc     wsock32:WSOCK32.dll
 0002:00000d68       __IMPORT_DESCRIPTOR_MFC42uD 5f605d68     MFC42UD:MFC42uD.DLL
 0002:00000d7c       __IMPORT_DESCRIPTOR_MSVCRTD 5f605d7c     msvcrtd:MSVCRTD.dll
 0002:00000d90       __IMPORT_DESCRIPTOR_KERNEL32 5f605d90     kernel32:KERNEL32.dll
 0002:00000da4       __IMPORT_DESCRIPTOR_USER32 5f605da4     user32:USER32.dll
 0002:00000db8       __NULL_IMPORT_DESCRIPTOR   5f605db8     MFC42UD:MFC42uD.DLL
 0003:00000000       ___xc_a                    5f607000     msvcrtd:cinitexe.obj
 0003:00000008       ___xc_z                    5f607008     msvcrtd:cinitexe.obj
 0003:0000000c       ___xi_a                    5f60700c     msvcrtd:cinitexe.obj
 0003:00000010       ___xi_z                    5f607010     msvcrtd:cinitexe.obj
 0003:0000002c       __pRawDllMain              5f60702c     dllnet.obj
 0003:00000030       ?_afxForceVectorDelete_mfcn@@3P6AXXZA 5f607030     dllnet.obj
 0003:00000038       ?GUID_ATLVer30@ATL@@3U_GUID@@A 5f607038     dllnet.obj
 0003:00000068       ??_R0?AVCNoTrackObject@@@8 5f607068     sockcore.obj
 0003:00000088       ??_R0?AV_AFX_SOCK_STATE@@@8 5f607088     sockcore.obj
 0003:000000a8       ??_R0?AVCObject@@@8        5f6070a8     sockcore.obj
 0003:000000c0       ??_R0?AVCAsyncSocket@@@8   5f6070c0     sockcore.obj
 0003:000000e0       ??_R0?AVCSocket@@@8        5f6070e0     sockcore.obj
 0003:000000f8       ??_R0PAVCException@@@8     5f6070f8     sockcore.obj
 0003:00000118       ??_R0?AVCFile@@@8          5f607118     sockcore.obj
 0003:00000130       ??_R0?AVCSocketFile@@@8    5f607130     sockcore.obj
 0003:00000150       ??_R0?AVCCmdTarget@@@8     5f607150     sockcore.obj
 0003:00000170       ??_R0?AVCWnd@@@8           5f607170     sockcore.obj
 0003:00000188       ??_R0?AVCSocketWnd@@@8     5f607188     sockcore.obj
 0003:000001b0       ??_R0?AVtype_info@@@8      5f6071b0     msvcrtd:ti_inst.obj
 0003:000001d0       __imp__WSAAsyncSelect@16   5f6071d0     wsock32:WSOCK32.dll
 0003:000001d4       __imp__WSAStartup@8        5f6071d4     wsock32:WSOCK32.dll
 0003:000001d8       __imp__WSASetLastError@4   5f6071d8     wsock32:WSOCK32.dll
 0003:000001dc       __imp__inet_ntoa@4         5f6071dc     wsock32:WSOCK32.dll
 0003:000001e0       __imp__ntohs@4             5f6071e0     wsock32:WSOCK32.dll
 0003:000001e4       __imp__accept@12           5f6071e4     wsock32:WSOCK32.dll
 0003:000001e8       __imp__htons@4             5f6071e8     wsock32:WSOCK32.dll
 0003:000001ec       __imp__inet_addr@4         5f6071ec     wsock32:WSOCK32.dll
 0003:000001f0       __imp__htonl@4             5f6071f0     wsock32:WSOCK32.dll
 0003:000001f4       __imp__closesocket@4       5f6071f4     wsock32:WSOCK32.dll
 0003:000001f8       __imp__gethostbyname@4     5f6071f8     wsock32:WSOCK32.dll
 0003:000001fc       __imp__recv@16             5f6071fc     wsock32:WSOCK32.dll
 0003:00000200       __imp__send@16             5f607200     wsock32:WSOCK32.dll
 0003:00000204       __imp__WSACleanup@0        5f607204     wsock32:WSOCK32.dll
 0003:00000208       __imp__WSAGetLastError@0   5f607208     wsock32:WSOCK32.dll
 0003:0000020c       __imp__socket@12           5f60720c     wsock32:WSOCK32.dll
 0003:00000210       __imp__recvfrom@24         5f607210     wsock32:WSOCK32.dll
 0003:00000214       __imp__sendto@24           5f607214     wsock32:WSOCK32.dll
 0003:00000218       __imp__connect@12          5f607218     wsock32:WSOCK32.dll
 0003:0000021c       __imp__getpeername@12      5f60721c     wsock32:WSOCK32.dll
 0003:00000220       __imp__getsockname@12      5f607220     wsock32:WSOCK32.dll
 0003:00000224       __imp__setsockopt@20       5f607224     wsock32:WSOCK32.dll
 0003:00000228       __imp__getsockopt@20       5f607228     wsock32:WSOCK32.dll
 0003:0000022c       __imp__bind@12             5f60722c     wsock32:WSOCK32.dll
 0003:00000230       __imp__ioctlsocket@12      5f607230     wsock32:WSOCK32.dll
 0003:00000234       __imp__listen@8            5f607234     wsock32:WSOCK32.dll
 0003:00000238       __imp__shutdown@8          5f607238     wsock32:WSOCK32.dll
 0003:0000023c       \177WSOCK32_NULL_THUNK_DATA_DLA 5f60723c     wsock32:WSOCK32.dll
 0003:00000240       ?ATL_CREATE_OBJECT@CComApartment@ATL@@2IA 5f607240     dllnet.obj
 0003:00000248       ?m_libid@CComModule@ATL@@2U_GUID@@A 5f607248     dllnet.obj
 0003:00000258       ?_pModule@ATL@@3PAVCComModule@1@A 5f607258     dllnet.obj
 0003:00000274       ?_afxSockState@@3V?$CProcessLocal@V_AFX_SOCK_STATE@@@@A 5f607274     sockcore.obj
 0003:0000027c       __hmod__WSOCK32            5f60727c     wsock32:WSOCK32.dll
 0003:00000280       ___puiHead                 5f607280     delayimp:delayhlp.obj
 0003:00000284       ___pfnDliFailureHook       5f607284     delayimp:delayhk1.obj
 0003:00000288       ___pfnDliNotifyHook        5f607288     delayimp:delayhk2.obj
 0003:0000028c       __adjust_fdiv              5f60728c     <common>
 0003:00000290       ___onexitend               5f607290     <common>
 0003:00000294       ___onexitbegin             5f607294     <common>

 entry point at        0001:000007c0

 Static symbols

 0001:0000105e       _$E375                     5f60205e f   sockcore.obj
 0001:0000106d       _$E372                     5f60206d f   sockcore.obj
 0001:00001072       _$E374                     5f602072 f   sockcore.obj
 0001:00001084       _$E373                     5f602084 f   sockcore.obj
 0001:000034f0       ?_AfxForceVectorDelete@@YAXXZ 5f6044f0 f   dllnet.obj
 0001:00000610       _$$$00001                  5f601610 f   msvcrtd:chkstk.obj
 0001:0000061c       probepages                 5f60161c f   msvcrtd:chkstk.obj
 0001:00000630       lastpage                   5f601630 f   msvcrtd:chkstk.obj
 0001:00000570       ?ArrayUnwindFilter@@YAHPAU_EXCEPTION_POINTERS@@@Z 5f601570 f   msvcrtd:ehvecdtr.obj
 0001:00000daf       ?OverlayIAT@@YGXPAU_IMAGE_THUNK_DATA32@@PBU1@@Z 5f601daf f   delayimp:delayhlp.obj

 33 bytes saved through ICF

